ASxxxx Linker V03.00/V05.40 + sdld,  page 1.
Hexadecimal  [32-Bits]

Area                                    Addr        Size        Decimal Bytes (Attributes)
--------------------------------        ----        ----        ------- ----- ------------
.  .ABS.                            00000000    00000000 =           0. bytes (ABS,CON)

      Value  Global                              Global Defined In Module
      -----  --------------------------------   ------------------------
     00000000  .__.ABS.                           _startup
     00000000  l_CABS                          
     00000000  l_DABS                          
     00000000  l_DATA                          
     00000000  l_INITIALIZED                   
     00000000  l_INITIALIZER                   
     00000000  l__CODE                         
     00000000  s_CABS                          
     00000000  s_DABS                          
     00000000  s__CODE                         
     00000001  l_SSEG                          
     00000001  s_DATA                          
     00000001  s_INITIALIZED                   
     00000001  s_SSEG                          
     00000003  l_GSFINAL                       
     0000000B  l_CONST                         
     00000023  l_GSINIT                        
     00000083  l_HOME                          
     00001205  l_CODE                          
     00008000  s_HOME                          
     00008083  s_GSINIT                        
     000080A6  s_GSFINAL                       
     000080A9  s_CONST                         
     000080B4  s_CODE                          
     000080B4  s_INITIALIZER                   

ASxxxx Linker V03.00/V05.40 + sdld,  page 2.
Hexadecimal  [32-Bits]

Area                                    Addr        Size        Decimal Bytes (Attributes)
--------------------------------        ----        ----        ------- ----- ------------
SSEG                                00000001    00000001 =           1. bytes (REL,CON)

      Value  Global                              Global Defined In Module
      -----  --------------------------------   ------------------------
ASxxxx Linker V03.00/V05.40 + sdld,  page 3.
Hexadecimal  [32-Bits]

Area                                    Addr        Size        Decimal Bytes (Attributes)
--------------------------------        ----        ----        ------- ----- ------------
HOME                                00008000    00000083 =         131. bytes (REL,CON)

      Value  Global                              Global Defined In Module
      -----  --------------------------------   ------------------------
ASxxxx Linker V03.00/V05.40 + sdld,  page 4.
Hexadecimal  [32-Bits]

Area                                    Addr        Size        Decimal Bytes (Attributes)
--------------------------------        ----        ----        ------- ----- ------------
GSINIT                              00008083    00000023 =          35. bytes (REL,CON)

      Value  Global                              Global Defined In Module
      -----  --------------------------------   ------------------------
ASxxxx Linker V03.00/V05.40 + sdld,  page 5.
Hexadecimal  [32-Bits]

Area                                    Addr        Size        Decimal Bytes (Attributes)
--------------------------------        ----        ----        ------- ----- ------------
GSFINAL                             000080A6    00000003 =           3. bytes (REL,CON)

      Value  Global                              Global Defined In Module
      -----  --------------------------------   ------------------------
ASxxxx Linker V03.00/V05.40 + sdld,  page 6.
Hexadecimal  [32-Bits]

Area                                    Addr        Size        Decimal Bytes (Attributes)
--------------------------------        ----        ----        ------- ----- ------------
CONST                               000080A9    0000000B =          11. bytes (REL,CON)

      Value  Global                              Global Defined In Module
      -----  --------------------------------   ------------------------
     000080AF  _SYSDivFactor                      stm8l15x_clk

ASxxxx Linker V03.00/V05.40 + sdld,  page 7.
Hexadecimal  [32-Bits]

Area                                    Addr        Size        Decimal Bytes (Attributes)
--------------------------------        ----        ----        ------- ----- ------------
CODE                                000080B4    00001205 =        4613. bytes (REL,CON)

      Value  Global                              Global Defined In Module
      -----  --------------------------------   ------------------------
     000080B4  _main                              main
     0000818F  _TRAP_IRQHandler                   stm8l15x_it
     00008190  _FLASH_IRQHandler                  stm8l15x_it
     00008191  _DMA1_CHANNEL0_1_IRQHandler        stm8l15x_it
     00008192  _DMA1_CHANNEL2_3_IRQHandler        stm8l15x_it
     00008193  _RTC_CSSLSE_IRQHandler             stm8l15x_it
     00008194  _EXTIE_F_PVD_IRQHandler            stm8l15x_it
     00008195  _EXTIB_G_IRQHandler                stm8l15x_it
     00008196  _EXTID_H_IRQHandler                stm8l15x_it
     00008197  _EXTI0_IRQHandler                  stm8l15x_it
     00008198  _EXTI1_IRQHandler                  stm8l15x_it
     00008199  _EXTI2_IRQHandler                  stm8l15x_it
     0000819A  _EXTI3_IRQHandler                  stm8l15x_it
     0000819B  _EXTI4_IRQHandler                  stm8l15x_it
     0000819C  _EXTI5_IRQHandler                  stm8l15x_it
     0000819D  _EXTI6_IRQHandler                  stm8l15x_it
     0000819E  _EXTI7_IRQHandler                  stm8l15x_it
     0000819F  _LCD_AES_IRQHandler                stm8l15x_it
     000081A0  _SWITCH_CSS_BREAK_DAC_IRQHandler   stm8l15x_it
     000081A1  _ADC1_COMP_IRQHandler              stm8l15x_it
     000081A2  _TIM2_UPD_OVF_TRG_BRK_USART2_TX_   stm8l15x_it
     000081A3  _TIM2_CC_USART2_RX_IRQHandler      stm8l15x_it
     000081A4  _TIM3_UPD_OVF_TRG_BRK_USART3_TX_   stm8l15x_it
     000081A5  _TIM3_CC_USART3_RX_IRQHandler      stm8l15x_it
     000081A6  _TIM1_UPD_OVF_TRG_COM_IRQHandler   stm8l15x_it
     000081A7  _TIM1_CC_IRQHandler                stm8l15x_it
     000081A8  _TIM4_UPD_OVF_TRG_IRQHandler       stm8l15x_it
     000081A9  _SPI1_IRQHandler                   stm8l15x_it
     000081AA  _USART1_TX_TIM5_UPD_OVF_TRG_BRK_   stm8l15x_it
     000081AB  _USART1_RX_TIM5_CC_IRQHandler      stm8l15x_it
     000081AC  _I2C1_SPI2_IRQHandler              stm8l15x_it
     000081AD  _USART_DeInit                      stm8l15x_usart
     000081C4  _USART_Init                        stm8l15x_usart
     00008241  _USART_ClockInit                   stm8l15x_usart
     0000827B  _USART_Cmd                         stm8l15x_usart
     00008290  _USART_SetPrescaler                stm8l15x_usart
     00008295  _USART_SendBreak                   stm8l15x_usart
     0000829D  _USART_ReceiveData8                stm8l15x_usart
     000082A0  _USART_ReceiveData9                stm8l15x_usart
     000082BB  _USART_SendData8                   stm8l15x_usart
     000082BE  _USART_SendData9                   stm8l15x_usart
     000082E3  _USART_ReceiverWakeUpCmd           stm8l15x_usart
     000082F8  _USART_SetAddress                  stm8l15x_usart
     00008307  _USART_WakeUpConfig                stm8l15x_usart
     00008316  _USART_HalfDuplexCmd               stm8l15x_usart
     0000832B  _USART_SmartCardCmd                stm8l15x_usart
     00008340  _USART_SmartCardNACKCmd            stm8l15x_usart
     00008355  _USART_SetGuardTime                stm8l15x_usart
     0000835A  _USART_IrDAConfig                  stm8l15x_usart
     0000836F  _USART_IrDACmd                     stm8l15x_usart
ASxxxx Linker V03.00/V05.40 + sdld,  page 8.
Hexadecimal  [32-Bits]

Area                                    Addr        Size        Decimal Bytes (Attributes)
--------------------------------        ----        ----        ------- ----- ------------
CODE                                000080B4    00001205 =        4613. bytes (REL,CON)

      Value  Global                              Global Defined In Module
      -----  --------------------------------   ------------------------
     00008384  _USART_DMACmd                      stm8l15x_usart
     0000839E  _USART_ITConfig                    stm8l15x_usart
     0000842D  _USART_GetFlagStatus               stm8l15x_usart
     00008455  _USART_ClearFlag                   stm8l15x_usart
     00008461  _USART_GetITStatus                 stm8l15x_usart
     000084F9  _USART_ClearITPendingBit           stm8l15x_usart
     00008502  _CLK_DeInit                        stm8l15x_clk
     00008543  _CLK_HSICmd                        stm8l15x_clk
     0000855B  _CLK_AdjustHSICalibrationValue     stm8l15x_clk
     00008567  _CLK_LSICmd                        stm8l15x_clk
     0000857F  _CLK_HSEConfig                     stm8l15x_clk
     00008594  _CLK_LSEConfig                     stm8l15x_clk
     000085A9  _CLK_ClockSecuritySystemEnable     stm8l15x_clk
     000085AE  _CLK_ClockSecuritySytemDeglitchC   stm8l15x_clk
     000085C6  _CLK_CCOConfig                     stm8l15x_clk
     000085CE  _CLK_SYSCLKSourceConfig            stm8l15x_clk
     000085D2  _CLK_GetSYSCLKSource               stm8l15x_clk
     000085D6  _CLK_GetClockFreq                  stm8l15x_clk
     00008629  _CLK_SYSCLKDivConfig               stm8l15x_clk
     0000862D  _CLK_SYSCLKSourceSwitchCmd         stm8l15x_clk
     00008645  _CLK_RTCClockConfig                stm8l15x_clk
     0000864D  _CLK_BEEPClockConfig               stm8l15x_clk
     00008651  _CLK_PeripheralClockConfig         stm8l15x_clk
     000086B9  _CLK_LSEClockSecuritySystemEnabl   stm8l15x_clk
     000086BE  _CLK_RTCCLKSwitchOnLSEFailureEna   stm8l15x_clk
     000086C3  _CLK_HaltConfig                    stm8l15x_clk
     000086E1  _CLK_MainRegulatorCmd              stm8l15x_clk
     000086F9  _CLK_ITConfig                      stm8l15x_clk
     0000875E  _CLK_GetFlagStatus                 stm8l15x_clk
     000087CC  _CLK_ClearFlag                     stm8l15x_clk
     000087D1  _CLK_GetITStatus                   stm8l15x_clk
     0000880B  _CLK_ClearITPendingBit             stm8l15x_clk
     0000881B  _GPIO_DeInit                       stm8l15x_gpio
     00008828  _GPIO_Init                         stm8l15x_gpio
     000088A3  _GPIO_ExternalPullUpConfig         stm8l15x_gpio
     000088BD  _GPIO_Write                        stm8l15x_gpio
     000088BF  _GPIO_WriteBit                     stm8l15x_gpio
     000088D6  _GPIO_SetBits                      stm8l15x_gpio
     000088DF  _GPIO_ResetBits                    stm8l15x_gpio
     000088EB  _GPIO_ToggleBits                   stm8l15x_gpio
     000088F4  _GPIO_ReadInputData                stm8l15x_gpio
     000088F7  _GPIO_ReadOutputData               stm8l15x_gpio
     000088F9  _GPIO_ReadInputDataBit             stm8l15x_gpio
     00008906  _GPIO_ReadOutputDataBit            stm8l15x_gpio
     00008912  _RTC_DeInit                        stm8l15x_rtc
     000089DD  _RTC_Init                          stm8l15x_rtc
     00008A26  _RTC_StructInit                    stm8l15x_rtc
     00008A36  _RTC_WriteProtectionCmd            stm8l15x_rtc
     00008A47  _RTC_EnterInitMode                 stm8l15x_rtc
     00008A68  _RTC_ExitInitMode                  stm8l15x_rtc
     00008A6D  _RTC_WaitForSynchro                stm8l15x_rtc
ASxxxx Linker V03.00/V05.40 + sdld,  page 9.
Hexadecimal  [32-Bits]

Area                                    Addr        Size        Decimal Bytes (Attributes)
--------------------------------        ----        ----        ------- ----- ------------
CODE                                000080B4    00001205 =        4613. bytes (REL,CON)

      Value  Global                              Global Defined In Module
      -----  --------------------------------   ------------------------
     00008A99  _RTC_RatioCmd                      stm8l15x_rtc
     00008ABD  _RTC_BypassShadowCmd               stm8l15x_rtc
     00008AE1  _RTC_SetTime                       stm8l15x_rtc
     00008B6D  _RTC_TimeStructInit                stm8l15x_rtc
     00008B7A  _RTC_GetTime                       stm8l15x_rtc
     00008BCC  _RTC_GetSubSecond                  stm8l15x_rtc
     00008BDD  _RTC_SetDate                       stm8l15x_rtc
     00008C84  _RTC_DateStructInit                stm8l15x_rtc
     00008C98  _RTC_GetDate                       stm8l15x_rtc
     00008CF1  _RTC_SetAlarm                      stm8l15x_rtc
     00008DE9  _RTC_AlarmStructInit               stm8l15x_rtc
     00008E03  _RTC_GetAlarm                      stm8l15x_rtc
     00008EB5  _RTC_AlarmCmd                      stm8l15x_rtc
     00008EFD  _RTC_AlarmSubSecondConfig          stm8l15x_rtc
     00008F38  _RTC_WakeUpClockConfig             stm8l15x_rtc
     00008F5D  _RTC_SetWakeUpCounter              stm8l15x_rtc
     00008F72  _RTC_GetWakeUpCounter              stm8l15x_rtc
     00008F80  _RTC_WakeUpCmd                     stm8l15x_rtc
     00008FBE  _RTC_DayLightSavingConfig          stm8l15x_rtc
     00008FE5  _RTC_GetStoreOperation             stm8l15x_rtc
     00008FEB  _RTC_OutputConfig                  stm8l15x_rtc
     00009012  _RTC_SynchroShiftConfig            stm8l15x_rtc
     0000904D  _RTC_SmoothCalibConfig             stm8l15x_rtc
     0000908F  _RTC_CalibOutputConfig             stm8l15x_rtc
     000090B3  _RTC_CalibOutputCmd                stm8l15x_rtc
     000090D7  _RTC_TamperLevelConfig             stm8l15x_rtc
     00009101  _RTC_TamperFilterConfig            stm8l15x_rtc
     00009122  _RTC_TamperSamplingFreqConfig      stm8l15x_rtc
     00009143  _RTC_TamperPinsPrechargeDuration   stm8l15x_rtc
     00009164  _RTC_TamperCmd                     stm8l15x_rtc
     0000918E  _RTC_ITConfig                      stm8l15x_rtc
     000091D6  _RTC_GetFlagStatus                 stm8l15x_rtc
     000091FB  _RTC_ClearFlag                     stm8l15x_rtc
     00009208  _RTC_GetITStatus                   stm8l15x_rtc
     0000922C  _RTC_ClearITPendingBit             stm8l15x_rtc
     0000925C  __divulong                         _divulong
     000092B7  ___sdcc_external_startup           _startup
ASxxxx Linker V03.00/V05.40 + sdld,  page 10.

Files Linked                              [ module(s) ]

../STM8L15X_LD/main.rel                   [ main ]
../STM8L15X_LD/stm8l15x_it.rel            [ stm8l15x_it ]
../STM8L15X_LD/stm8l15x_usart.rel         [ stm8l15x_usart ]
../STM8L15X_LD/stm8l15x_clk.rel           [ stm8l15x_clk ]
../STM8L15X_LD/stm8l15x_gpio.rel          [ stm8l15x_gpio ]
../STM8L15X_LD/stm8l15x_rtc.rel           [ stm8l15x_rtc ]


Libraries Linked                          [ object file ]

/opt/sdcc/bin/../share/sdcc/lib/stm8/stm8.lib
                                          [ _divulong.rel ]
/opt/sdcc/bin/../share/sdcc/lib/stm8/stm8.lib
                                          [ _startup.rel ]

ASxxxx Linker V03.00/V05.40 + sdld,  page 11.

User Base Address Definitions

HOME = 0x8000
DATA = 0x0001

